:020000040000FA
:0600000080284B300130A6
:080008000000200080310C19FA
:10001000122820000B14200095019A309600B2019E
:10002000B017532820000B102000901A1E28B1177B
:10003000260A03193117B11930284B28B113B11909
:100040002D28311F4B28B11A4B28AA01A901A8015C
:10005000A701A601B101B1165328F030B10553280C
:1000600030149030B1052608AF002708AE002808EC
:10007000AD0029080319AD0103192808AC002A08AE
:10008000AB00031D5328AC1F53282808AC002908D7
:10009000AB00AD015328310DA60DA70DA80DA90D7C
:0C00A000AA0DB11AB10A1010901209004C
:10010000203085000030840000301A00F0300402F6
:10011000031C8428402321000C308C058E01200014
:100120008C018E01003022009101930100303100DA
:100130009B00003021009D0021009E000030230024
:100140008C00003022008C00003024008C00003035
:1001500027008C0002303D009500003023008E0007
:10016000003022008E00003024008E000030270076
:100170008E0003303D00A0000D303D00A1000E3088
:100180003D00A2000F303D00A30014303D00A4004C
:100190000C303D00A500FF3021008E008330200090
:1001A0009700403020009800013020009B00003074
:1001B00020009C00013028009300003028009400AB
:1001C000003028009A00003028009B001F302000DB
:1001D0009E009F30250093000030250091000430E0
:1001E000250092009F3025009700003025009500E3
:1001F0000C30250096009F3026009300003026002A
:1002000091000630260092009F30260097000030B3
:10021000260095001E3026009600043020009F0026
:100220000730280097007F3028009E00003025000E
:100230009F0080302C00990000302C009700803007
:100240002C009C0000302C009A00243021009700E4
:10025000A63023009E00803023009D00183023002C
:100260009F00003023009C00423023009B000C3094
:1002700021008C00C03021008E0001302100900050
:1002800002303C009000003021009100003021003D
:1002900092000030210093000030210094000030D3
:1002A00020008B0020003F24950199019A019001C4
:1002B00091019201930194018B176400B01B642992
:1002C000131E6A29B101B201B0131312E1302800E4
:1002D000920020007B2130187D2133181B10331829
:1002E0005D291B14C022B608031D79298D3109250B
:1002F000813105255D296400080030108C3100240F
:10030000813133180800C330B0052D08031D97292B
:10031000FF302C020319080040302E06C0390319A3
:10032000301680302E06C03903193015A0293F3011
:100330002D020319B016DE302D06FE390319B01553
:100340003C303006031908002B082C062D062E061B
:100350002F02031D080030100130F0008B137030A5
:1003600085003030700784000008A5002030700739
:1003700084000008A4001030700784000008A30067
:100380000030700784000008A2008B1722082B029F
:10039000031DAA2A23082C02031DAA2A0130700279
:1003A000031DF3293019EA29B019052AB01AE129E9
:1003B000AE1AB022AE1EB4222E081F39F600F61770
:1003C0000800AE1FB022AE1BB4222E087F39F60003
:1003D000F617080080302E06E039031DF3292E1E83
:1003E000BC222E1AB8223019F829B019052A0800A3
:1003F000AE1E2E1225082E06F039031DAA2A250846
:100400002E050F390319552A0D2A24082D02031D24
:10041000AA2A25082E050319552A01307002031D4A
:10042000162A7318162A7314B01499230230700216
:10043000031D1F2AF3181F2AF314B014A823033036
:100440007002031D282A7319282A7315B014B723C4
:1004500004307002031D312AF319312AF315B01448
:10046000C62305307002031D3A2A731A3A2A7316FE
:10047000B014D52306307002031D432AF31A432A11
:10048000F316B014E42307307002031D4C2A731BCB
:100490004C2A7317B014F32308307002031D552A39
:1004A000F31B552AF317B014F923B01D5C2A2E094B
:1004B00025050319AA2A612A2E0925050F390319D2
:1004C000AA2A01307002031D6A2A731C6A2A73105B
:1004D000B014FF2302307002031D732AF31C732A29
:1004E000F310B014072403307002031D7C2A731D1F
:1004F0007C2A7311B0140D2404307002031D852A68
:10050000F31D852AF311B014132405307002031D66
:100510008E2A731E8E2A7312B014192406307002AC
:10052000031D972AF31E972AF312B0141F240730D5
:100530007002031DA02A731FA02A7313B014252470
:1005400008307002031DA92AF31FA92AF313B0145F
:100550002B24AA2AF00A0930700203180800AE29D9
:10056000751BB01475130800751FB01475170800BB
:10057000F51FB014F5170800F51BB014F5130800AB
:10058000B01C0800B0101030F2007308F100CE2249
:100590003030F2007508F100CE220800703085007E
:1005A0007208840000087102031908003100710804
:1005B00093007208910070309200151715158B1377
:1005C00055309600AA30960095148B17151120000F
:1005D0008B1371083100151593002000720831004B
:1005E000910055309600AA30960095146400951835
:0A05F000F62A151120008B170800F1
:1006800010303124F30030303124F5006230312451
:10069000F7006330312477020319B3166D3031242B
:1006A000E1006118F3016118F501B0303124210037
:1006B000A0002000B13031242100A1002000B23080
:1006C00031242100A2002000B33031242100A300F6
:1006D0002000B43031242100A4002000B5303124A2
:1006E0002100A5002000B63031242100A600200002
:1006F000B73031242100A7002000B8303124210078
:10070000A8002000B93031242100A9002000BA300F
:1007100031242100AA002000BB3031242100AB008D
:100720002000BC3031242100BE000319BE0A200085
:100730000800C4303124D000031D4E14661C08008C
:10074000733031242100D0005C14200042140800D2
:10075000C5303124D100031DCE14671C080073304E
:1007600031242100D100DC142000C2140800C6305E
:100770003124D200031D4E15681C0800733031244B
:100780002100D2005C15200042150800C73031243A
:10079000D300031DCE15691C0800733031242100DD
:1007A000D300DC152000C2150800C8303124D40065
:1007B000031D4E166A1C0800733031242100D4003A
:1007C0005C16200042160800C9303124D500031DF4
:1007D000CE166B1C0800733031242100D500DC16C6
:1007E0002000C2160800AC3031242100BC042000D7
:1007F0000800AD3031242100BC04200008000C1694
:10080000CA303124D600031D4F140C120800CB301F
:100810003124D700031DCF140800CC303124D80078
:10082000031D4F150800CD303124D900031DCF150D
:100830000800CE303124DA00031D4F160800CF30F7
:100840003124DB00031DCF160800AC303824210012
:10085000BC0520000800AD3038242100BC05200074
:100860000800F2007030850072088400000808005B
:10087000F200703085007208840000090800D00181
:10088000D101D201D3010800DC1B4B2C73085D059C
:100890000319812C532C751F502C5C1F532C7E2C5C
:1008A0005C1B532C7E2C5C185C2CDC18602C5C19B7
:1008B000632CDC1B5D2C732C732CF51B732C812C8F
:1008C0005E18702C7E2CDE1C7E2C21006908200016
:1008D0005D05031D08005D082100E9042000702C5F
:1008E0005D08C00408005D084E05031D08005D0892
:1008F000C00408005D082100E90420005D09C0056E
:1009000008005D084F05031D08005D09C0050800CB
:10091000331E0800203085002200200884000008D3
:1009200023009A002200A00AAB302002A130031855
:10093000A0002000080064303124B900E01EB90195
:100940006530E01E60303124BA002200A130A000E2
:100950007730A100AD30A2002000AD303A1CAF309E
:10096000BA1C40382200A3002000AD303A1DAF3041
:10097000BA1D40382200A4002000AD303A1EAF302E
:10098000BA1E40382200A5002000AD303A1FAF301B
:10099000BA1F40382200A6002000AD30391CAF300D
:1009A000B91C40382200A7002000AD30391DAF30FF
:1009B000B91D40382200A8002000AD30391EAF30EC
:1009C000B91E40382200A90020008330F700F70349
:1009D000AD30771CAF30F71C40382200AA00200051
:1009E00022002309A2062409A2062509A206260937
:1009F000A2062709A2062809A2062909A2062A0991
:100A0000A206AD30A20420000800921B40258824D5
:100A1000DD015D146608DC004424DD01DD14670897
:100A2000DC004424DD015D156808DC004424DD01A0
:100A3000DD156908DC004424DD015D166A08DC0070
:100A40004424DD01DD166B08DC004424C626142690
:100A5000921C080092108025172766183C2620005B
:100A600067185326200068186A2620006918812616
:100A700020006A18812620006B18812620000800BB
:100A80009213CE01D008031D4E14D108031DCE14BD
:100A9000D208031D4E15D308031DCE15D408031D1F
:100AA0004E16D508031DCE16CF01D608031D4F14D0
:100AB000D708031DCF14D808031D4F15D908031DEF
:100AC000CF15DA08031D4F16DB08031DCF164E188D
:100AD000D003CE18D1034E19D203CE19D3034E1A28
:100AE000D403CE1AD5034F18D603CF18D7034F1906
:100AF000D803CF19D9034F1ADA03CF1ADB03080042
:100B000042082100DC05200020004008F8002000F9
:100B1000210020083C182108B6002208BC18230830
:100B2000B70024083C192508B8002608BC19270876
:100B3000B90028083C1A2908BA002A08BC1A2B0850
:100B4000BB0003105C18B60C0310DC18B70C0310C4
:100B50005C19B80C0310DC19B90C03105C1ABA0C40
:100B60000310DC1ABB0C781CB601F81CB701781D09
:100B7000B801F81DB901781EBA01F81EBB01BD0B02
:100B8000FA2D3E08BD002100300836020319CD2D94
:100B90000318CC2DB003CD2DB00A3108370203194C
:100BA000D62D0318D52DB103D62DB10A320838023F
:100BB0000319DF2D0318DE2DB203DF2DB20A33082F
:100BC00039020319E82D0318E72DB303E82DB30A02
:100BD00034083A020319F12D0318F02DB403F12D56
:100BE000B40A35083B020319FA2D0318F92DB50391
:100BF000FA2DB50A210030082500920021003108A5
:100C000025009600210032082600920021003308BA
:100C100026009600210034082C0098002100350899
:100C20002C009B002000080021004108C00029265C
:100C3000C1004208C0002926C2004308C000411C70
:100C40002926C3004408C000C11C2926C400200076
:100C500008002100C501C0080319C003401845144D
:100C6000C01A45144508C501401C4514C01E451452
:100C7000C505C50C400C08004E180800421C0800B1
:100C80002100D60B08004108D600D003200003192C
:100C900042102100C1185C1444195C14C31E5C147A
:100CA000C21D5C100800CE180800C21C08002100FC
:100CB000D70B08004308D700D10320000319C21046
:100CC0002100411ADC14441BDC14431DDC14421CBB
:100CD000DC1008004E190800421D08002100D80B46
:100CE00008004208D800D203200003194211210055
:100CF000C11A5C15C21B5C15C31D5C15441C5C113C
:100D00000800CE190800C21D08002100D90B0800F8
:100D10004408D900D30320000319C211210043194C
:100D2000DC154119DC15421EDC15C41FDC1108005E
:100D30004E1A0800421E08002100DA0B0800410983
:100D4000DA00D403200003194212210042195C1674
:100D5000441B5C16C31D5C16411E5C120800CE1AB3
:100D60000800C21E08002100DB0B08004409DB005C
:100D7000D50320000319C21221004318DC16C11943
:100D8000DC16C21EDC16C41FDC1208002100E103C1
:100D90002000031D0800F61FEF2E0310761A03141F
:100DA000F60D1F30F605F6132100630820007602C9
:100DB000031CE22E0319EF2E76082100E300E00069
:100DC0002000EF2E76082100E300200021006608B5
:100DD0000319E007200021006408E2002000210040
:100DE00065086307600220000318092F5E10E618EB
:100DF0004010E718C010E8184011E918C011EA18AF
:100E000040120130210063076002200003180A2FFE
:100E100008005E142100E2032000031D08002100E9
:100E20006408E20020002100E00320000800210007
:100E3000E8032000031D08002100E815E703200057
:100E4000031D0800703085007A30840000082100FE
:100E5000E7002000DE1C2E2FDE1008002100E90133
:060E60002000DE14080072
:101800003318192C2D080319072CB60108002E08CF
:1018100003190C2CB60108002C080319112CB60171
:1018200008003010B60A02303602031C08003314D8
:1018300008008C0130102B082C062D062E062F02D6
:101840000319232C08007C302C06FC3903198A2C40
:10185000331178302C06FC390319422C74302C06D5
:10186000FC3903197D2C2C08031D3D2C2D08031D6C
:101870003D2C2E08031D3D2C08003310B6013312F9
:10188000092508002E08BC00E0303C06E039031DA5
:1018900008000130BC180430B80003103C18B80D23
:1018A0003C19B80E8C31A6248C31BA248C313C1AE8
:1018B000652CB31E0800350838050319622CBC19C5
:1018C000C8240800BC1DC8240800331F08000730C6
:1018D0002D0203190800BC1D702C3808B504722CA9
:1018E0003809B5058B133408F2003508F100823150
:1018F000CE228C318B17C8240800B31E08008C310F
:10190000A6248C31BA248C3135082E02031D080020
:10191000C82408003319A42C8C31A6248C31331F21
:101920000800B3190800B4080319912D07302D02DF
:10193000031908008B133408F2002E08F1008231DD
:10194000CE228C318B173315C82408003313B31AF9
:1019500033170F302D0203193317B3152C18080055
:10196000AC1808008E31F8268C31B400B408031D81
:10197000B3110800B501B3190800703085003408B0
:1019800084000008B500340340300319B500080096
:101990000C1628009801443099001A1420001412E3
:1019A0006400141ED02C141228001A1020000C12EF
:1019B00008006A30B4008A253508E0007A30B400A7
:1019C0008A2535082100E70020007B30B4008A25F5
:1019D00035082100E40020007C30B4008A25350859
:1019E0002100E50020007D30B4008A253508210063
:1019F000E60020002030870046308600A630B40084
:101A00008A2535081E00B40A50300602031C002D3A
:101A10000800331A08003316D92484319B248D31F1
:101A20000130B7003708913EB4008A253508BB0065
:101A30006430BB080319232DBB0388303B18023EDA
:101A4000BB18043EBB0AB4008A253508B900BB08A0
:101A5000031D2C2DE01EB9016530E01E6030BB086F
:101A60000319392DBB0389303B18023EBB18043ED5
:101A7000BB0AB4008A253508BA003708003EB40016
:101A80008A253908B50203194D2D8B13F10034084E
:101A9000F2008231CE228D318B173708103EB40010
:101AA0008A253A08B50203195D2D8B13F10034081D
:101AB000F2008231CE228D318B179B303707B40074
:101AC0008A253508B900B1253708203EB4008A259B
:101AD0003908B5020319742D8B13F1003408F20094
:101AE0008231CE228D318B173708303EB4008A25E3
:101AF0003A08B5020319842D8B13F1003408F20063
:101B00008231CE228D318B17B70A09303702031884
:101B10000800122D70308500340884000008B500DC
:101B20000800B7016030B4007030850034088400CC
:101B30000008B5003708BD008E3130268D31B50262
:101B40000319AA2D8B13F1003408F2008231CE2242
:101B50008D318B17B70A503037020319C82CB40ADD
:101B6000942D0130BA00B90303103918BA0DB91811
:101B7000BA0DB918BA0DB90CB90CB90A3919CE2D6C
:101B8000BA173030B918BA0439183A123919DE3098
:101B9000B918DF30391D0301B90008003918BA0E31
:021BA000C62D50
:101C60000E308A003D0882070334503401340134B9
:101C7000C034033400340034003400340034003401
:101C80000034003400340034003402340F34403463
:101C9000FF34FF34FF34FF34FF34FF342034043486
:101CA00004341034FF34FF34FF34FF34FF34013484
:101CB000FF34FF34FF34FF34003400340034003488
:101CC0000034003400340034003400340034003474
:101CD0000034003400340034003400340034003464
:101CE0000134023403340434053406340734083430
:101CF00009340A34003400348034C03400340034F1
:101D000003340C34003400342034053420340534DA
:101D1000203405342034053420340534203405348F
:101D20000A34FF34FF34FF34FF34FF34FF34FF3410
:101D300001340134013401340134013401340134FB
:101D40000134013401340134FF34FF34FF34FF34F3
:101D5000FF34FF34FF34FF34FF34FF34FF34FF34EB
:101D6000FF34FF34FF34FF34FF34FF34FF34FF34DB
:101D7000FF34FF34FF34FF34FF34FF34FF34FF34CB
:101D8000FF34FF34FF34FF34FF34FF34FF34FF34BB
:101D9000FF34FF34FF34FF34FF34FF34FF34FF34AB
:081DA000FF34FF34FF34FF346F
:081DF0000F308A002D0882006B
:101E00006034003400340034003400346134013470
:101E1000003400340034003400340034623463345D
:101E200064346534663467346834693400340034AB
:101E300000340034003400346A346B34003400342D
:101E400000340034003400340034003400340034F2
:101E50000034003400340034003400346C346D3409
:101E60006E346F3470347134723473347434753446
:101E700076347734783479347A347B347C347D34F6
:101E800000340034003400340034003400340034B2
:101E900000340034003400340034003400340034A2
:101EA0000034003400340034003400340034003492
:101EB0000034003400340034003400340034003482
:101EC0000034003400340034003400340034003472
:101ED0007E347F34003400340034003400348034E5
:101EE000813482348334843485348634873488342E
:101EF00089348A348B348C348D348E348F349034DE
:101F0000913492349334943495349634973498348D
:101F100099349A349B349C349D349E349F34A0343D
:101F2000A134A234A334A434A534A634A734A834ED
:101F3000A934AA34AB34AC34AD34AE34AF34B0349D
:101F4000B134B234B334B434B534B634B734B8344D
:101F5000B934BA34BB34BC34BD34BE34BF34C034FD
:101F6000C134C234C334C434C534C634C734C834AD
:101F7000C934CA34CB34CC34CD34CE34CF34D0345D
:101F8000D134D234D334D434D534D634D734D8340D
:101F9000D934DA34DB34DC34DD34DE34DF34E034BD
:101FA000E134E234E334E434E534E634E734E8346D
:101FB000E934EA34EB34EC34ED34EE34EF34F0341D
:101FC000F134F234F334F434F534F634F734F834CD
:101FD000F934FA34FB34FC34FD34FE34FF3400347D
:101FE0000034003400340034003400340034003451
:101FF0000034003400340034003400340034003441
:020000040001F9
:08000000800000000000000078
:02000E008C174D
:060010003C25FF1FFF3F2D
:10E00000010000000000000000000000000000000F
:10E010000000000000000000000000000000000000
:10E0200000000300030003000300030003000300DB
:10E0300003000300030003000300030003000300C8
:10E0400000000000000000000000000000000000D0
:10E0500000000000000000000000DE00DE00DE0026
:10E0600000008100820084008800B100B200B4008A
:10E07000B800A100A200A400A80001000200040052
:10E08000FF00FF00FF00FF00FF00FF00FF00FF0098
:10E09000FF00FF00FF00FF00FF00FF00FF00FF0088
:10E0A000FF00FF00FF00FF00FF00FF00FF00FF0078
:10E0B000FF00FF00FF00FF00FF00FF00FF00FF0068
:10E0C0000300500001000100C00003000000000038
:10E0D0000000000000000000000000000000000040
:10E0E000000002000F004000FF00FF00FF00FF00E3
:10E0F000FF00FF002000040004001000FF00FF00EC
:10E10000FF00FF00FF000100FF00FF00FF00FF0015
:10E1100000000000000000000000000000000000FF
:10E1200000000000000000000000000000000000EF
:10E1300000000000000000000100020003000400D5
:10E14000050006000700080009000A0000000000A2
:10E150008000C0000000000003000C000000000070
:10E16000200005002000050020000500200005001B
:10E1700020000500200005000A00FF00FF00FF004E
:10E18000FF00FF00FF00FF0001000100010001008F
:10E190000100010001000100010001000100010077
:10E1A000FF00FF00FF00FF00FF00FF00FF00FF0077
:10E1B000FF00FF00FF00FF00FF00FF00FF00FF0067
:10E1C000FF00FF00FF00FF00FF00FF00FF00FF0057
:10E1D000FF00FF00FF00FF00FF00FF00FF00FF0047
:10E1E000FF00FF00FF00FF00FF00FF00FF00FF0037
:10E1F000FF00FF00FF00FF00FF00FF00FF00FF0027
:00000001FF
